:020000040000FA
:04000000EC303A287E
:040004000034003490
:08000800A000030EA100831209
:100010008B1C32288B1032181428B21C3228643002
:10002000010203183128182800001628172818285C
:1000300019281A281B281C281D281E281F283210A2
:10004000B214A810031005190314AA0DA90DA80DC8
:10005000B10B322832152A08AF002908AE00280853
:10006000AD00B21081010B11210E8300A00E200EF5
:02007000090085
:0C007400203084008001840A80300402E7
:10008000031C3C281230B1001D2283160C3085055C
:1000900087018312850187010730990000309A009B
:1000A000103083168E008312603083168F00831207
:1000B00000308316910000008312C830831681003F
:1000C000831231309000003083168C008312103080
:1000D0008B00432381018E018F010B118B100B10BC
:1000E0008C018B17812032199720B40B7F280310C5
:1000F00085190314BA0DF0303A0203196721AA23B7
:1001000072286400321808000B1D08000B11B21091
:1001100032141230B100051D9228331483160113D6
:10012000831208003310831601178312080032115E
:100130000130B7008B1320303707371A313E831652
:100140009B001C141A088312A400A500C030A50649
:1001500010303707371A313E83169B001C141A08DB
:100160008312A30000303707371A313E83169B00F5
:100170001C141A088312A2008B17331CC5282209ED
:100180000339A200A309A409A50922082D02031D11
:10019000612923082E02031D612924082F02031D53
:1001A000612901303702031DDA283E18DA283E148F
:1001B0003F14382202303702031DE328BE18E3281B
:1001C000BE143F14442203303702031DEC283E19AD
:1001D000EC283E153F14502204303702031DF52849
:1001E000BE19F528BE153F145C2205303702031DE9
:1001F000FE283E1AFE283E163F14682206303702BB
:10020000031D0729BE1A0729BE163F1474220730A2
:100210003702031D10293E1B10293E173F14802270
:1002200008303702031D1929BE1B1929BE173F14B8
:100230008C2209303702031D22295E1822295E1400
:100240003F1497220A303702031D2B29DE182B2971
:10025000DE143F14A2220B303702031D34295E192D
:1002600034295E153F14AD220C303702031D3D29A1
:10027000DE193D29DE153F14B8220D303702031D6B
:1002800046295E1A46295E163F14C3220E303702F5
:10029000031D4F29DE1A4F29DE163F14CE220F30E0
:1002A0003702031D58295E1B58295E173F14D922B7
:1002B00010303702031D6129DE1B6129DE173F1450
:1002C000E422B70A0F303702031808009A280130D9
:1002D000B600B400B500B70085018701B213402312
:1002E0008120B40B8029031085190314BA0DF03056
:1002F0003A020319AD29B50B80299630B500B92112
:10030000321D70293211331C8A292D090339AD00A1
:10031000AE09AF092F1CB2132F1C7029B21B702914
:100320002E187029B2178B1320303707371A313E39
:10033000BC002F08BB00082210303707371A313EA7
:10034000BC002E08BB00082200303707371A313EA8
:10035000BC002D08BB0008228B1785018701B70A56
:10036000B6010130B5000F303702031C702943235A
:100370000800013037020319F02202303702031956
:10038000F522033037020319FA2204303702031929
:10039000FF22053037020319042306303702031900
:1003A00009230730370203190E23083037020319D7
:1003B000132309303702031918230A3037020319AF
:1003C0001D230B303702031922230C303702031987
:1003D00027230D30370203192C230E30370203195F
:1003E00031230F3037020319362310303702031937
:1003F0003B2308003F1C08003F101030BC003E08A3
:10040000BB0008223030BC005E08BB000822080098
:100410008B133B0883161C159A0083123C08831625
:100420009B0055309D00AA309D009C1464009C18D0
:10043000162A1C1183128B170800831610309B009C
:100440001C141A088312BE00831630309B001C1443
:100450001A088312DE00FF30C800CA15CB15CC1570
:10046000CD15CE15CF15D015D115D215D315080041
:100470008130BE05FF30DE050230C405C00000300B
:10048000C200C6005F1008008230BE05FF30DE05E6
:100490000230C405C0000230C200C6005F10080070
:1004A0008430BE05FF30DE050430C405C0000030D6
:1004B000C200C6005F1008008830BE05FF30DE05B0
:1004C0000530C405C0000030C200C6005F1008003F
:1004D0009030BE05FF30DE050430C405C000043096
:1004E000C200C6005F100800A030BE05FF30DE0568
:1004F0001030C405C0000030C200C6005F10080004
:10050000C030BE05FF30DE051830C405C000003025
:10051000C200C6005F100800FF30BE050030DE05D7
:100520001030C505C1000030C300C70008007F308F
:10053000BE050130DE051030C505C1001030C30016
:10054000C70008007F30BE050230DE052030C5053B
:10055000C1000030C300C70008007F30BE05043072
:10056000DE052830C505C1000030C300C700080003
:100570007F30BE050830DE052030C505C1002030C3
:10058000C300C70008007F30BE051030DE05803094
:10059000C505C1000030C300C70008007F30BE059C
:1005A0002030DE05C030C505C1000030C300C700E3
:1005B00008007F30BE054030DE050030C505C100B3
:1005C0000030C300C70008007F30BE058030DE0564
:1005D0000030C505C1000030C300C7000800080096
:1005E0002030850600308706080020308506003060
:1005F00087060800013085060030870608001130A4
:100600008506003087060800013085060030870621
:100610000800003085060230870608000230850693
:100620000230870608000030850601308706080082
:10063000003085060130870608000030850620302E
:100640008706080000308506243087060800003041
:1006500085062030870608000030850608308706AA
:10066000080000308506183087060800003085062F
:100670000030870608000030850600308706080035
:100680003E18F02208003E183822BE1844223E19B7
:100690005022BE195C223E1A6822BE1A74223E1BEA
:1006A0008022BE1B8C225E189722DE18A2225E19C1
:1006B000AD22DE19B8225E1AC322DE1ACE225E1BDC
:1006C000D922DE1BE4220800B601B401B5013D1CAD
:1006D0006C2BBD01BD146E2BBD013D143D08B60051
:1006E0006400722B732B742B752B762BFF30B51B8C
:1006F0008500B51F8501B40B702BB50B702B031053
:10070000B60CB608031D702B0030BC003D08BB00C2
:100710000822080005125C180516DC1C8512DC187E
:1007200085165C1D05105C190514DC1D8510DC198F
:1007300085145C1E87105C1A8714DC1E0711DC1AF6
:1007400007155C1F07105C1B0714DC1F8712DC1BDE
:10075000871608008F08031908008F0178308E0073
:10076000C80FE82DC80ADF19DC2B441CDC2B461C03
:10077000CD2BCA1CBE2BCA014A15EA2B4A1DC32B1E
:10078000CA01CA15EA2BCA1DC82BCA014A16EA2B90
:100790004A1EEA2BCA01CA14EA2B4A1DD22BCA01EF
:1007A0004A16EA2BCA1DD72BCA014A16EA2B4A1E43
:1007B000EA2BCA01CA14EA2BCA1CE12BCA014A154A
:1007C000EA2B4A1DE62BCA01CA15EA2B4A1EEA2B60
:1007D000CA014A15DF19132CC41C132CC61C042C87
:1007E000CB1CF52BCB014B15212C4B1DFA2BCB0130
:1007F000CB15212CCB1DFF2BCB014B16212C4B1ED7
:10080000212CCB01CB14212C4B1D092CCB014B16D9
:10081000212CCB1D0E2CCB014B16212C4B1E212C39
:10082000CB01CB14212CCB1C182CCB014B15212C2C
:100830004B1D1D2CCB01CB15212C4B1E212CCB018C
:100840004B15DF194A2C441D4A2C461D3B2CCC1C51
:100850002C2CCC014C15582C4C1D312CCC01CC151A
:10086000582CCC1D362CCC014C16582C4C1E582C18
:10087000CC01CC14582C4C1D402CCC014C16582CBF
:10088000CC1D452CCC014C16582C4C1E582CCC01A0
:10089000CC14582CCC1C4F2CCC014C15582C4C1D76
:1008A000542CCC01CC15582C4C1E582CCC014C157A
:1008B000DF19822CC41D822CC61D732CCD1C642C08
:1008C000CD014D155F13902C4D1D692CCD01CD151B
:1008D000902CCD1D6E2CCD014D16902C4D1E902CC4
:1008E000CD01CD14902C4D1D782CCD014D16902CA2
:1008F000CD1D7D2CCD014D16902C4D1E902CCD0183
:10090000CD14902CCD1C872CCD014D15902C4D1D58
:100910008C2CCD01CD15902C4D1E902CCD014D155C
:10092000DF19BB2C5F1BBB2C441EBB2C461EAC2C02
:10093000CE1C9D2CCE014E15C92C4E1DA22CCE01D5
:10094000CE15C92CCE1DA72CCE014E16C92C4E1E7D
:10095000C92CCE01CE14C92C4E1DB12CCE014E1681
:10096000C92CCE1DB62CCE014E16C92C4E1EC92C3C
:10097000CE01CE14C92CCE1CC02CCE014E15C92CD4
:100980004E1DC52CCE01CE15C92C4E1EC92CCE0134
:100990004E15DF19F22CC51DF22CC71DE32CCF1C00
:1009A000D42CCF014F15002D4F1DD92CCF01CF15C1
:1009B000002DCF1DDE2CCF014F16002D4F1E002D18
:1009C000CF01CF14002D4F1DE82CCF014F16002D65
:1009D000CF1DED2CCF014F16002D4F1E002DCF0146
:1009E000CF14002DCF1CF72CCF014F15002D4F1D1C
:1009F000FC2CCF01CF15002D4F1E002DCF014F1520
:100A0000DF19292D451E292D471E1A2DD01C0B2D0F
:100A1000D0015015372D501D102DD001D015372D78
:100A2000D01D152DD0015016372D501E372DD00159
:100A3000D014372D501D1F2DD0015016372DD01D2D
:100A4000242DD0015016372D501E372DD001D01433
:100A5000372DD01C2E2DD0015015372D501D332D84
:100A6000D001D015372D501E372DD0015015DF196C
:100A7000602DC51E602DC71E512DD11C422DD101E8
:100A800051156E2D511D472DD101D1156E2DD11D42
:100A90004C2DD10151166E2D511E6E2DD101D11448
:100AA0006E2D511D562DD10151166E2DD11D5B2D70
:100AB000D10151166E2D511E6E2DD101D1146E2D06
:100AC000D11C652DD10151156E2D511D6A2DD101FD
:100AD000D1156E2D511E6E2DD1015115DF19982D96
:100AE000451F982D471F892DD21C7A2DD2015215F2
:100AF000DF13A62D521D7F2DD201D215A62DD21D9A
:100B0000842DD2015216A62D521EA62DD201D2142A
:100B1000A62D521D8E2DD2015216A62DD21D932D1B
:100B2000D2015216A62D521EA62DD201D214A62DE8
:100B3000D21C9D2DD2015215A62D521DA22DD201DF
:100B4000D215A62D521EA62DD2015215DF19D12D78
:100B5000DF1BD12DC51FD12DC71FC22DD31CB32D17
:100B6000D3015315DF2D531DB82DD301D315DF2D20
:100B7000D31DBD2DD3015316DF2D531EDF2DD30101
:100B8000D314DF2D531DC72DD3015316DF2DD31DD5
:100B9000CC2DD3015316DF2D531EDF2DD301D314DB
:100BA000DF2DD31CD62DD3015315DF2D531DDB2D87
:100BB000D301D315DF2D531EDF2DD3015315FA2199
:100BC0004008C4004108C5005F18DF145F1CDF1037
:100BD0004808C9000C304A05031D05120C304B05AE
:100BE000031D85120C304C05031D05100C304D05FE
:100BF000031D85100C304E05031D87100C304F056A
:100C0000031D07110C305005031D07100C30510552
:100C1000031D87120C305205031D07120C305305BB
:100C2000031D871149080E020318422E12304A058F
:100C3000031D051612304B05031D851612304C0599
:100C4000031D051412304D05031D851412304E0589
:100C5000031D871412304F05031D07151230500570
:100C6000031D071412305105031D8716123052055B
:100C7000031D071612305305031D8715FF30480268
:100C8000031908008F08031D0800812049080E027F
:100C9000031C422E18304A05031D051206304A0572
:100CA000031D051618304B05031D851206304B0534
:100CB000031D851618304C05031D051006304C0524
:100CC000031D051418304D05031D851006304D0514
:100CD000031D851418304E05031D871006304E0580
:100CE000031D871418304F05031D071106304F05EB
:100CF000031D071518305005031D07100630500559
:100D0000031D071418305105031D871206305105C5
:100D1000031D871618305205031D071206305205B1
:100D2000031D071618305305031D871106305305A0
:060D3000031D87150800F9
:084000000C00030007000100A1
:02400E00CC33B1
:10420000010003000300030003000200020002009B
:104210000200000000000000000003000300030093
:10422000810000000000000000000000000000000D
:104230000000C000C000C000C000C000C000C0003E
:10424000FF00C300F300CF00FF00C300F300CF0066
:10425000FF00C300F300CF00FF00C300F300CF0056
:104260000000FF00FF00FF00FF00FF00FF00FF0055
:10427000FF00FF00FF00FF00FF00FF00FF00FF0046
:10428000FF000300FF00FF00FF00FF00FF00FF0032
:10429000FF00FF00FF00FF00FF00FF00FF00FF0026
:1042A000FF00C000FF00FF00FF00FF00FF00FF0055
:1042B000FF00FF00FF00FF00FF00FF00FF00FF0006
:1042C000FF00FF00FF00FF00FF00FF00FF00FF00F6
:1042D000FF00FF00FF00FF00FF00FF00FF00FF00E6
:1042E000FF00FF00FF00FF00FF00FF00FF00FF00D6
:1042F000FF00FF00FF00FF00FF00FF00FF00AA001B
:00000001FF
